:040000008A15002835
:0C000600000000000000000000000800E6
:0E001200533083120313FD00FD0B0D28080070
:10002000243083120313FC00B530FD00FD0B1628AD
:0A003000FC0B162800000000080079
:10003A0083120313F801F9011030FC00710DF80D59
:10004A00F90D7408F8027508031C750FF9020318F4
:10005A0035287408F80775080318750FF90703108F
:0A006A00F00DF10DFC0B2328080037
:1000740083120317BD1B40288611412886153D1B9A
:100084004528061146280615BD1A4A2886104B280D
:1000940086143D1A4F28061050280614831603139D
:1000A4006F185728831206165928831206128616CB
:1000B400032086120317BD1961288611622886154C
:1000C4003D196628061167280615BD186B28861089
:1000D4006C2886143D18702806107128061483169F
:1000E40003136F187828831206167A2883120612CF
:1000F40086160320861283166F1C822810208328FC
:0401040009200800C6
:0E010800F201F101F001F801F30100300800EE
:100116007B15FB1F95280130F300F201F101F00178
:08012600FA0DF20CFF30080095
:08012E00FA1FF2130030080073
:100136007B14FB1FA628F201FA1FFF30F200F10024
:0A014600F000FA0DF20CFF30080083
:10015000FB14FB1FB228FF30F300F200F100F000A7
:08016000FA0DF20CFF3008005B
:0E016800831203172E088A002D08820008005B
:1001760083120317BB0105303B020318C9283B084D
:100186003A07840020308000BB0ABE283B083A07A5
:1001960084008001BB033B083A07BC000A30F40028
:1001A600F5013808F0003908F1001D207808F00044
:1001B6007908F1003030F00703173C088400700816
:1001C60080000A30F400F5013808F0003908F10023
:1001D6001D2070080317B8007108B90000307106B9
:1001E600031DF72800307006031DFA28FC28BB0300
:0401F600CE28080007
:1001FA00A0017208031D12297108F2007008F100AB
:10020A00F001A0157208031D12297108F200F1010C
:10021A00A01120167208031920292008F302031DD1
:10022A00031C24290310F21B2829F00DF10DF20DED
:10023A00F30B182924290130FC0084202B290230D1
:0E024A00FC008B202B290430FC0097200800BC
:10025800831603136F10831203173808BD003A2062
:0602680083166F1408006C
:10026E0083120313FB01FA01F9018030F800F10C3F
:10027E00F00C031C4B297408F90775080318750F49
:10028E00FA070318FB0A0310F01F53297408FA0724
:10029E0075080318750FFB07FB0CFA0CF90CF80C1C
:1002AE00031C3E297B08F3007A08F2007908F1005E
:0602BE007808F0000800C2
:1002C400710DF80DF90D7408F8027508031C750F0B
:1002D400F902F00DF10D0F30FC00710DF80DF90D60
:1002E4007408701C7B29F8027508031C750FF90249
:1002F4008029F80775080318750FF907F00DF10D3B
:10030400FC0B6F2970188C297408F80775080318FA
:08031400750FF9070000080055
:10031C00243083120313FD00FD0B9229000008000A
:10032C00831203131A08F100981C9E291812181630
:06033C007108F00008004A
:1003420083120313FB017308031D77080319F829AD
:1003520072087606FA007708F3077E30031CB52987
:10036200F3020318FB29B829F302031CFE297208C1
:10037200F8007108FC007008FD00F817F61703106A
:10038200F201F101F0011830A0007D1CD22974089D
:10039200F00775080318750FF10776080318760F32
:1003A200F207F20CF10CF00CF80CFC0CFD0C031033
:1003B200A00BC629F21BE229F80DF00DF10DF20D8A
:1003C200F3037B1B701CF429F81FF429F00A0319AC
:1003D200F10A0319F20A031DF429F20CF10CF00CD4
:1003E200F30A0319FB29FA1FF2130030002A013025
:1003F2008420002A0230A820002A04308B2000002A
:020402000800F0
:1004040083120313FB01730803193F2A7208FA00CD
:10041400F2178E30F302F31F422AF309F30A08306D
:100424007302031C252AF300F10D7208F100F20196
:1004340008307302031C252AF300F10DF10173083F
:10044400031D03102D2A730803192D2A0310F20C1F
:10045400F10CF30B282A7B1B711C372A031C372A47
:10046400F10A0319F20AF21B4E2AFA1F512AF20961
:10047400F109F10A0319F20A512AF201F101512A90
:100484007B14FB1F542AF201FA1F542AFF30F20096
:10049400F100FA0DF20C542A0130FC00562A003007
:1004A400FC00562AFF30FC00FC0803195A2A9B2042
:0A04B4007108F0007208F100080062
:0E04BE000030831203138C1A0130F000080086
:1004CC00831203137008F8007108F000F101F201B7
:1004DC00F301FB01FC019630F300FA01F01F7C2ABA
:1004EC00F809F009F80A0319F00AFA177008F10074
:0C04FC007808F000F801F201FD20080073
:10050800831603131208013EF000F1010318F10AE3
:10051800831203172F08F400F50137210630F20083
:100528007008F4007108F50072080319A02AF50C88
:10053800F40CF513FF3E992A0430F1007408F0001A
:1005480071080319AB2AF00D7010FF3EA52A303050
:100558007005F3007408F0007508F100F10CF00C58
:10056800F113F10CF00CF113700895000F3097059A
:060578007308970408005F
:10057E00831203137408003A031DCE2A7508003A3D
:10058E00031DCE2AFF30F0007F30F100272B83129F
:10059E000313FD01F901F801710870040319003409
:1005AE0071087506FA00FA1BFD09FB01F51FE42A16
:1005BE00F409F509F40A0319F50AF11FEB2AF009FB
:1005CE00F109F00A0319F10A71087504FA00FA1B11
:1005DE00002B62217B18132BFD1F0034F009F1094B
:1005EE00F00A0319F10AF809F909F80A0319F90AC8
:1005FE000034F51F0F2BF11B0B2B7108F90070083F
:10060E00F800F101F001F32AF101F001F00A0034D3
:10061E00F109F009FB0AF02AF80A0319F90A74081D
:10062E007802031DF32A75087902031DF32AF901D6
:10063E00F801F00A0319F10AF11FF32A0000FF3442
:02064E000800A2
:10065000831203139F01C0309F046F09F0007008DC
:1006600083169F051F179F17831203172F08F0008B
:10067000F00D7010F00D7010F00D70107008031375
:100680009F041F148E211F151F1D482B0000442B93
:100690001F101E08F100F00183161E08F004003040
:0406A000F104080059
:1006A40083160313981690308312980083168717C5
:1006B400071383128C1E612B1A08F0005B2B0800B1
:1006C400FF30831203179E00FF309F00FF30A0000D
:1006D400FF3003139F01C0309F046F09F0007008BE
:0E06E40083169F051F179F1783121F1408000F
:1006F200B4208A110A128000840AAD0A0319AE0AD4
:08070200F003031D792B080030
:0C070A00831203139501171297120800C8
:100716009D2B803083120317AF00B02BC030AF0083
:10072600B02B9430AF00B02BD430AF00B02B80305C
:10073600AF00B02B831203172F08013A03198C2B35
:100746002F08023A0319912B2F08033A0319942B09
:100756002F08043A0319972B9A2B3003F0002F0821
:10076600F0077008AF007008BD003A2083166F10BE
:1007760083120317B20132083107840000080319F7
:10078600CE2B3208310784000008B8002C218312D2
:0E0796000317B20ABE2B831603136F1408005C
:1007A40083120317B401B5012F08B6003008B7004F
:1007B40080303006F00080307002031DE32B0030DF
:1007C4002F020318F12B0130B4000030B5002F08BC
:1007D400003CB6003008031C013EB701B7023608DE
:1007E400B8003708B9003108BA00BB200630B2009F
:1007F4000030B3003308003C031D022C3208003CD7
:1008040003181D2C32083107F20001303202F000C7
:100814000030031C013E3302F100700831078400EC
:100824000008F00072088400700880000130B202F1
:10083400031CB303FC2B31088400203080003408EF
:10084400350403193B2CB201B3013208310784008B
:100854000008203A031D322CB20A0319B30A272CCC
:100864000130B202031CB3033208310784002D3077
:0408740080000800F8
:1008780083160313861206120610861006118611B7
:100888008312861206128611061186100610102091
:1008980010201020861406148616032086121020B5
:1008A8008616032086121020861603208612102032
:1008B800061086160320861210208616032086123C
:1008C80086108615861603208612102086110614B7
:1008D800861603208612061086160320861210201C
:1008E8008616032086120614861603208612102008
:1008F8000610861603208612861506158614061419
:0E090800861603208612102083166F14080036
:10091600831603130711831212150C30970408006F
:100A600021308400473083120313F00093300317C2
:100A7000AD000430AE007923A03084000D30831225
:100A8000F0001A300317AD000530AE00792368304E
:100A9000840008308312F00027300317AD000530C2
:100AA000AE007923AD30840040308312F000DA309C
:0C0AB0000317AD000430AE0079230800ED
:101000008A1130258A1583120317940195019201E4
:10101000930190019101960197019C019D019A0114
:101020009B019801990183160313ED01EE01081449
:101030008814081588150711831212149210F930BC
:10104000831692008A1185238A158A118B248A15AA
:1010500081308316990018158A1152238A158A1136
:1010600062238A158A113C248A150C3083120317D7
:10107000BD008A113A208A1501300317AF000330F2
:10108000B0002D30B1008A118B238A1502308312F3
:101090000317AF000330B0002130B1008A118B2359
:1010A0008A150D30FB00AF30FC00B630FD00FD0BA3
:1010B0005728FC0B5728FB0B5728000001308312E0
:1010C0000317BD008A113A208A1503138818722865
:1010D000003003171306031D6F2801301206031991
:1010E0007228462903170130AF000130B0003E30AE
:1010F000B1008A118B238A15023083120317AF00C7
:101100000130B0003530B1008A118B238A15881068
:1011100083128814081C4629013003179000003000
:1011200091000130BD008A113A208A150130031761
:10113000AF000130B000BC30B1008A118B238A159A
:10114000831203171008110403194629AF018A11ED
:1011500028238A15700883120317A3007108A400BE
:101160001830F4000030F5008A1137218A15700814
:101170000317A3007108A4006430F4000030F500E8
:101180008A11BF228A1570080317A3007108A400F2
:101190007008AF008A1184228A1503172308A10062
:1011A0002408A2002308F0002408F1008A11662216
:1011B0008A158530F400EB30F5005130F6007D30B3
:1011C000F7008A11A1218A158A1102228A15700856
:1011D0000317A1007108A2007008AF007108B000E9
:1011E0002530B1008A11D2238A150230AF000130B8
:1011F000B0002530B1008A118B238A154130FC00E4
:10120000EE30FD00FD0B0229FC0B022900008312C9
:10121000081D26298316881483128810031790014D
:10122000910192019301AF018A1184228A15413004
:10123000FC00EE30FD00FD0B1B29FC0B1B29000000
:1012400001300317BD008A113A208A15881D4529EF
:1012500003179001910183160313881483128810D9
:10126000013003179600003097009201930101307E
:10127000BD008A113A208A154130FC00EE30FD0095
:10128000FD0B4029FC0B40290000A02803138819FE
:101290005029031716081704031D5029F10152297C
:1012A0000130F1007108013A031D772B031701305B
:1012B000AF000130B000E230B1008A118B238A15F3
:1012C000023083120317AF000130B000D930B100F3
:1012D0008A118B238A150330FB008A30FC005530BD
:1012E000FD00FD0B7129FC0B7129FB0B712900001E
:1012F0000000013083120317BD008A113A208A15BD
:101300000317A301A40101309C0000309D000317C6
:101310001C081D040319772B8A1196218A15700861
:10132000323A03199D29003083166E06031D9A294F
:1013300001306D0603199D29532B013083120317C9
:101340009400003095000317140815040319532B5B
:101350008A115F228A157008013A031D3A2B8A11FF
:1013600096218A157008613A031D762A19300317F1
:101370002307F00024080318013EF1007008A300C1
:101380007108A4007008AF008A1184228A1503171F
:101390002308A1002408A2002308F0002408F1007B
:1013A0008A1166228A15CD30F400CC30F5004C301D
:1013B000F6007D30F7008A11A1218A158A110222D8
:1013C0008A1570080317A1007108A2007008AF0009
:1013D0007108B0002530B1008A11D2238A1501307E
:1013E000AF000130B000CA30B1008A118B238A15DA
:1013F000023083120317AF000330B0002530B10074
:101400008A118B238A150030831203172406031DCB
:101410000B2AFA302306031D762A0130BD008A11FB
:101420003A208A15013003179A0000309B000317F9
:101430001A081B040319762AFA30AF008A11842295
:101440008A1501300317AF000130B000AD30B10094
:101450008A118B238A15023083120317AF000330E1
:10146000B000A030B1008A118B238A158A11962111
:101470008A157008623A031D462A01300317BD0021
:101480008A113A208A1503179A019B010313881CBD
:101490005B2A03179A019B01960197019C019D010C
:1014A0000130920000309300940195010130BD009D
:1014B0008A113A208A158A1196218A157008333AC2
:1014C000031D752A0317AF018A1184228A15031799
:1014D0009A019B01960197019C019D019401950140
:1014E0000130BD008A113A208A15172A8A119621E7
:1014F0008A157008623A031D3A2B1930031723022C
:10150000F0000030031C013E2402F1007008A3002B
:101510007108A4007008AF008A1184228A1503178D
:101520002308A1002408A2002308F0002408F100E9
:101530008A1166228A15CD30F400CC30F5004C308B
:10154000F6007D30F7008A11A1218A158A11022246
:101550008A1570080317A1007108A2007008AF0077
:101560007108B0002530B1008A11D2238A150130EC
:10157000AF000130B0005930B1008A118B238A15B9
:10158000023083120317AF000330B0002530B100E2
:101590008A118B238A150030831203172406031D3A
:1015A000D32A00302306031D3A2B01309800003067
:1015B00099000130BD008A113A208A1503171808D6
:1015C000190403193A2BAF018A1184228A150130BC
:1015D0000317AF000130B0004A30B1008A118B23ED
:1015E0008A15023083120317AF000330B000683051
:1015F000B1008A118B238A158A1196218A157008E9
:10160000613A031D0B2B0317980199010130BD00AE
:101610008A113A208A15881C1F2B031798019901FB
:10162000960197019C019D010130920000309300CA
:10163000940195010130BD008A113A208A158A1162
:1016400096218A157008333A031D392B0317AF0111
:101650008A1184228A15031798019901960197012E
:101660009C019D01940195010130BD008A113A2031
:101670008A15DE2A8A1196218A157008333A031DCD
:10168000522B0317AF018A1184228A150317960182
:1016900097019C019D01940195010130BD008A11C3
:1016A0003A208A15A3298312881C642B03179601FC
:1016B00097019C019D0101309200003093000130A0
:1016C000BD008A113A208A158A1196218A15700860
:1016D000323A031D762B01308316ED000030EE0008
:1016E0000130831203179C0000309D008729652874
:0216F000782B55
:100926004234493445344E34563445344E344934D1
:0809360044344F345334003403
:10093E00203420342034433454344434423400348C
:10094E0041344334543449345634413444344F34AE
:02095E00003463
:100960004D344F3444344F3420344D3441344E34BC
:08097000553441344C340034CD
:100978002034203420342034563465346C346F34B9
:0E0988006334693464346134643420340034E0
:100996002034203420342034563465346C346F349B
:0E09A6006334693464346134643420340034C2
:1009B4002034203420342034563465346C346F347D
:0E09C4006334693464346134643420340034A4
:1009D2002034203420342034563465346C346F345F
:0C09E200633469346434613464340034DC
:1009EE002034203420342034563465346C346F3443
:0E09FE0063346934643461346434203400346A
:100A0C0041346334743469347634613464346F340F
:020A1C000034A4
:100A1E004134553454344F344D34413454344934C4
:060A2E0043344F34003494
:100A340020342034203420342034313430343034E1
:0A0A44002034203420342034003424
:0E0A4E0020342034203420342034303400345E
:020A5C000F3455
:02400E004A2F37
:00000001FF
